:0400000063EF00F0BA
:060008004D823CEF0DF0FB
:100018004D80D8CF13F0E8CF14F0E0CF15F0FACF29
:1000280016F0FBCF17F0E9CF18F0EACF19F0E1CFBF
:100038001AF0E2CF1BF0D9CF1CF0DACF1DF0F3CFC6
:100048001EF0F4CF1FF0F6CF20F0F7CF21F0F8CF55
:1000580022F0F5CF23F04DC024F04EC025F04FC05C
:1000680026F050C027F027C050F026C04FF025C01A
:100078004EF024C04DF023C0F5FF22C0F8FF21C088
:10008800F7FF20C0F6FF1FC0F4FF1EC0F3FF1DC01E
:10009800DAFF1CC0D9FF1BC0E2FF1AC0E1FF19C07C
:1000A800EAFF18C0E9FF17C0FBFF16C0FAFF15C02A
:1000B800E0FF14C0E8FF13C0D8FF4D90100027EFF1
:1000C8000EF0899400F000F000F000F000F000F06D
:1000D80000F000F000F000F000F000F000F000F098
:1000E80000F000F000F000F000F000F000F000F088
:1000F80000F000F000F000F000F000F000F000F078
:1001080000F000F000F000F000F000F000F000F067
:1008980000F000F0898400F000F000F000F000F0B3
:1008A80000F000F000F000F000F000F000F000F0C0
:1008B80000F000F000F000F000F000F000F000F0B0
:1008C80000F000F000F000F000F000F000F000F0A0
:1008D80000F000F000F000F000F000F000F000F090
:1010680000F000F000F08994860E0001C46FFE0EB7
:10107800C56F020EC66FEFEC0FF084B0FED78B0E73
:101088000001C46FFF0EC56F010EC66FEFEC0FF0C5
:10109800A20E0001C46FFE0EC56F020EC66FEFEC04
:1010A8000FF0300E4FEC11F08B0E0001C46FFF0EE5
:1010B800C56F010EC66FEFEC0FF0860E0001C46F0E
:1010C800FE0EC56F020EC66FEFEC0FF084B0FED7B0
:1010D8008B0E0001C46FFF0EC56F010EC66FEFECDB
:1010E8000FF089841200D00E00019525D46FD56BBE
:1010F800FF0ED5239651D00FD66F9751D00FD76FCB
:101108009851D00FD86FD651640DF3CFD1F0F4CFEA
:10111800D2F0D7510A0DF350D127F450D223D85129
:10112800D125E36F000ED221E46F1DD1E3C0C7F0D3
:10113800D451BFEC0CF01200310E00019519D8A45F
:1011480006D0E3C0C7F0070EBFEC0CF01200320E59
:1011580000019519D8A406D0E3C0C7F0060EBFEC6D
:101168000CF01200330E00019519D8A41200E3C048
:10117800C7F0050EBFEC0CF01200E3C0C3F0E4C0EA
:10118800C4F0000E0001C66F0A0EC56FEDEC10F03A
:1011980000019951D16FD26BC351D127C451D223C9
:1011A800D00ED125E16FFF0ED221E26F310E9519D5
:1011B800D8A408D0E1C0CAF0E2C0CBF0010EE7EC39
:1011C8000DF01200320E00019519D8A408D0E1C024
:1011D800CAF0E2C0CBF0020EE7EC0DF01200330EBD
:1011E80000019519D8A41200E1C0CAF0E2C0CBF002
:1011F800020EE7EC0DF01200310E00019519D8A48B
:1012080006D0010EC76F040EBFEC0CF01200000EE2
:101218000001C76F040EBFEC0CF01200310E000184
:101228009519D8A406D0010EC76F030EBFEC0CF0B9
:101238001200000E0001C76F030EBFEC0CF0120085
:10124800310E00019519D8A412009651D16F97510B
:10125800DF6FD1C0E0F01F0EDF15DD6FDE6BDDC084
:10126800D1F0DEC0D2F0D890D137D237D890D1376C
:10127800D237D890D137D237D1C0DDF0D2C0DEF026
:10128800DFC0D1F0E0C0D2F0060ED36FD890D233D1
:10129800D133D32FFBD71F0ED115DB6FDC6BDBC02F
:1012A800D1F0DCC0D2F0D890D137D237D890D1372E
:1012B800D237D890D137D237D1C0DBF0D2C0DCF0EA
:1012C800DFC0D1F0E0C0D2F00B0ED36FD890D2338C
:1012D800D133D32FFBD71F0ED115D96FDA6BD9C0F5
:1012E800D1F0DAC0D2F0D890D137D237D890D137F0
:1012F800D237D890D137D237D1C0D9F0D2C0DAF0AE
:10130800310E9819D8A416D0D9C0CAF0DAC0CBF0DB
:10131800010E28EC0FF0DBC0CAF0DCC0CBF0020EE7
:1013280028EC0FF0DDC0CAF0DEC0CBF0030E28ECCD
:101338000FF01200000E0001CB6F000ECA6F010EF5
:1013480028EC0FF0000E0001CB6F000ECA6F020EE2
:1013580028EC0FF0000E0001CB6F000ECA6F030ED1
:1013680028EC0FF0120000019451440AD8B405D7B4
:10137800020AD8B453D70A0AD8B4DED6030AD8B4B6
:10138800D5D61D0AD8B45CD7010AD8A4120034D720
:10139800000E0001D16F0F0ED16501D02ED0D151B2
:1013A800010D600EF324D96E000EF420DA6E000EE3
:1013B800DF6ED151010D800EF324D96E010EF42099
:1013C800DA6E010EDF6ED151020D700EF324D96E64
:1013D800000EF420DA6E000EDE6E000EDD6ED151C6
:1013E800020D900EF324D96E010EF420DA6E010E70
:1013F800DE6E000EDD6ED12BCED7000EC46F1F0E31
:10140800C56F800EB0EC10F0FE0E0001C46F030E25
:10141800C56F800EB0EC10F0000E0001C46F0F0E07
:10142800C56F800EB0EC10F0010E0001C46F140EF1
:10143800C56F800EB0EC10F0000E0001C86F000EF2
:10144800C76F000E66EC0EF0000E0001C86F000EAC
:10145800C76F010E66EC0EF0000E0001C86F000E9B
:10146800C76F020E66EC0EF0000E0001C86F000E8A
:10147800C76F030E66EC0EF0000E0001C86F000E79
:10148800C76F040E66EC0EF0000E0001C86F000E68
:10149800C76F050E66EC0EF0000E0001C76F000E58
:1014A800BFEC0CF0000E0001C76F010EBFEC0CF092
:1014B800000E0001C76F020EBFEC0CF0000E000119
:1014C800C76F030EBFEC0CF0000E0001C76F040ECF
:1014D800BFEC0CF0000E0001C76F050EBFEC0CF05E
:1014E800000E0001C76F060EBFEC0CF0000E0001E5
:1014F800C76F070EBFEC0CF0000E0001C46F000EA2
:10150800C56F400EB0EC10F0010E0001C46F000E64
:10151800C56F400EB0EC10F0020E0001C46F000E53
:10152800C56F400EB0EC10F0030E0001C46F000E42
:10153800C56F400EB0EC10F0040E0001C46F000E31
:10154800C56F400EB0EC10F0050E0001C46FB10E6F
:10155800C56F400EB0EC10F0060E0001C46F000E0F
:10156800C56F400EB0EC10F0070E0001C46F000EFE
:10157800C56F400EB0EC10F0080E0001C46F000EED
:10158800C56F400EB0EC10F00A0E0001C46FFF0EDC
:10159800C56F400EB0EC10F0100E0001C46F000EC5
:1015A800C56F400EB0EC10F0110E0001C46F000EB4
:1015B800C56F400EB0EC10F0120E0001C46F000EA3
:1015C800C56F400EB0EC10F0130E0001C46F000E92
:1015D800C56F400EB0EC10F0140E0001C46F000E81
:1015E800C56F400EB0EC10F0150E0001C46FB00EC0
:1015F800C56F400EB0EC10F0160E0001C46F000E5F
:10160800C56F400EB0EC10F0170E0001C46F000E4D
:10161800C56F400EB0EC10F0180E0001C46F000E3C
:10162800C56F400EB0EC10F01A0E0001C46FFF0E2B
:10163800C56F400EB0EC10F012000001C76F080E25
:101648000001C56F0B0E01EC11F0000E0001C56F13
:101658000C0E01EC11F039D0210E0001C56F0D0EF2
:1016680001EC11F0620E0001C56F0E0E01EC11F0D5
:10167800760E0001C56F0F0E01EC11F031D0220E6D
:101688000001C56F0D0E01EC11F0B10E0001C56F20
:101698000E0E01EC11F03B0E0001C56F0F0E01ECB0
:1016A80011F01ED0100E0001C56F0D0E01EC11F0E7
:1016B800A70E0001C56F0E0E01EC11F0620E0001BD
:1016C800C56F0F0E01EC11F00BD00001C751000AD5
:1016D800D8B4D5D7010AD8B4E5D7030AD8B4BCD74B
:1016E8005B0E0001C56F100E01EC11F0F80E000141
:1016F800C56F110E01EC11F0030E0001C56F120E3B
:1017080001EC11F0220E0001C56F130E01EC11F06F
:10171800F80E0001C56F140E01EC11F0000E000167
:10172800C56F0A0E01EC11F0470E0001C56F150ECA
:1017380001EC11F0B60E0001C56F210E01EC11F09D
:10174800100E0001C56F220E01EC11F0180E0001F9
:10175800C56F180E01EC11F01D0E0001C56F190EB2
:1017680001EC11F01C0E0001C56F1A0E01EC11F00E
:10177800C70E0001C56F1B0E01EC11F0000E000131
:10178800C56F1C0E01EC11F0B20E0001C56F1D0EE5
:1017980001EC11F0EA0E0001C56F230E01EC11F007
:1017A8002A0E0001C56F240E01EC11F0000E000195
:1017B800C56F250E01EC11F0110E0001C56F260E44
:1017C80001EC11F0590E0001C56F290E01EC11F062
:1017D800810E0001C56F2C0E01EC11F0350E0001D1
:1017E800C56F2D0E01EC11F0090E0001C56F2E0E0C
:1017F80001EC11F00B0E0001C56F000E01EC11F0A9
:10180800070E0001C56F020E01EC11F0040E000175
:10181800C56F070E01EC11F0050E0001C56F080E2B
:1018280001EC11F0000E0001C56F090E01EC11F07A
:101838003D0E0001C56F060E01EC11F01200000EFE
:101848000001E76F010EE66F000EE96F000EE86F0A
:101858000A0EEB6FCD0EEA6F0A0EED6FAA0EEC6F53
:10186800A1EC0EF027EC10F05F0E0001C46FFE0E25
:10187800C56F010EC66FEFEC0FF001EC0FF070ECC6
:1018880011F00009D8B45ED00D0E0001C46FFF0E30
:10189800C56F020EC66FEFEC0FF08BA402D0010EDD
:1018A80001D0000E00080001E56F010EE527E547AD
:1018B800E5478B50E519FB0BE5198B6E940ECC6F41
:1018C800000ECD6FD8EC0EF0660E0001C46FFF0E4F
:1018D800C56F010EC66FEFEC0FF0000E0001EF6F41
:1018E800000EEE6FEF5114E10A0EEE5DD8B010D085
:1018F800940EEE25D96E000EEF21DA6EDF5097ECCC
:101908000FF0200E97EC0FF00001EE4BEF2BEAD70B
:1019180062EC11F0FA0E0001C46FFE0EC56F020EE4
:10192800C66FEFEC0FF077EC08F0660E0001C46F9D
:10193800FF0EC56F010EC66FEFEC0FF083EC11F0D0
:101948007FEC11F000019305D8A402D0000E936F2C
:101958009205D8A407D0000E926F90510008E56F49
:10196800E529906F9105D8A488D72AEC11F0000ECC
:101978000001916F82D70001CD6F0001C7510008A7
:10198800C86FC829C76F1A0EC46F400EB5EC0FF0A8
:101998000001D06FCF6B0A0EC46F400EB5EC0FF08C
:1019A8000001C86FCF51C811CF6FD051D06FCDC0D3
:1019B800C8F0010EC96F000ECA6FC82B03D0D890AB
:1019C800C937CA37C82FFBD70001C91DCB6FCA1D3D
:1019D800CC6FCF51CB15CF6FD051CC15D06FCDC0B8
:1019E800C8F0C751C96FCA6BC82B03D0D890C93784
:1019F800CA37C82FFBD70001CF51C911CF6FD051BB
:101A0800CA11D06F000ECE6F0F0ECE6501D020D058
:101A1800CEC0C8F0010EC96F000ECA6FC82B03D024
:101A2800D890C937CA37C82FFBD70001CF51C9137F
:101A3800D051CA13CE51020D900EF324D96E010E67
:101A4800F420DA6EC9C0DEFFCAC0DDFFCE2BDCD7BA
:101A58000A0EC46FCFC0C5F0400EB0EC10F01A0EDD
:101A68000001C46FD051C56F400EB0EC10F01200E9
:101A7800FACF01F0FBCF02F0E9CF03F0EACF04F090
:101A8800E1CF05F0E2CF06F0D9CF07F0DACF08F0C2
:101A9800F3CF09F0F4CF0AF0F6CF0BF0F7CF0CF044
:101AA800F8CF0DF0F5CF0EF04DC00FF04EC010F08E
:101AB8004FC011F050C012F0F2BAF2A408D0B10E23
:101AC800D76EE00ED66E010E3A6EF2940DD0A3B822
:101AD800A4A804D058EC10F0A49806D0A3BAA4AADD
:101AE80003D085EC10F0A49A12C050F011C04FF04A
:101AF80010C04EF00FC04DF00EC0F5FF0DC0F8FF3E
:101B08000CC0F7FF0BC0F6FF0AC0F4FF09C0F3FFD3
:101B180008C0DAFF07C0D9FF06C0E2FF05C0E1FF31
:101B280004C0EAFF03C0E9FF02C0FBFF01C0FAFFDF
:101B38004D92110089848D828D94D20E0001C46F5C
:101B4800FE0EC56F010EC66FEFEC0FF065EC00F0EE
:101B58008D0E0001C46FFF0EC56F010EC66FEFEC4E
:101B68000FF0BD0E0001C46FFE0EC56F000EC66FEC
:101B7800EFEC0FF0010E21EC0BF08D0E0001C46F9D
:101B8800FF0EC56F010EC66FEFEC0FF0E60E0001F9
:101B9800C46FFE0EC56F000EC66FEFEC0FF0440E5B
:101BA8000001C56F000EC66F080EC76F3E0E73ECBE
:101BB8000FF08D0E0001C46FFF0EC56F010EC66FCA
:101BC800EFEC0FF012000001CC6F0F0E0001CE6F8A
:101BD800CD692DD0CDC0C7F0CEC0C8F00A0E66ECD6
:101BE8000EF0CAC0C7F0CBC0C8F00B0E66EC0EF002
:101BF8001200CDC0C7F0CEC0C8F0080E66EC0EF0DB
:101C0800CAC0C7F0CBC0C8F0090E66EC0EF01200CF
:101C1800CDC0C7F0CEC0C8F00C0E66EC0EF0CAC03E
:101C2800C7F0CBC0C8F00D0E66EC0EF01200000134
:101C3800CC51010AD8B4CED7030AD8B4DAD7010AEE
:101C4800D8A41200E5D7B40EF66E220EF76E000E79
:101C5800F86E00EEF0F010EE10F00900F5CFEEFF90
:101C6800E550E150FAE1F60EF66E220EF76E000E20
:101C7800F86E00EE44F010EE08F00900F5CFEEFF24
:101C8800E550E150FAE102EE00F0820EEE6AE80655
:101C9800FDE101EE00F0DF0EEE6AE806FDE100EE80
:101CA80060F0630EEE6AE806FDE100EE28F01C0E17
:101CB800EE6AE806FDE14D904D92000EF86E0001C7
:101CC80023EF0CF00001C96F0001C951020D700E1D
:101CD800F324D96E000EF420DA6EC7C0DEFFC8C048
:101CE800DDFFC945E846FC0B060FC46F000EC56F43
:101CF800800EB0EC10F00001C945E846FC0B070F58
:101D0800C46F000EC56F800EB0EC10F00001C9451D
:101D1800E846FC0B080FC46FC7C0C5F0800EB0ECD6
:101D280010F00001C945E846FC0B090FC46FC85103
:101D3800C56F800EB0EC10F01200D388D38AD38C14
:101D4800FC0ED316000ED26E000ED16E000EC26EBF
:101D5800E70E0F01486F0B0E496F000E896E000EDB
:101D68008A6E000E8B6E000E8C6E000E8D6E958640
:101D780095946FEC10F08C9E8C8C959E959C95821A
:101D8800958043EC11F094948B841DEC11F09680AF
:101D9800969496929294928292808D848D82898470
:101DA800D08EF28EF28C12003B0EC5EC10F00001C2
:101DB800CE6F7F0ECE17D8B41CD03F0ED9EC10F0E2
:101DC8000001D16FCCC0C6F0CDC0C7F0D1C0C8F0FB
:101DD8003F0E4FEC0FF0CF0E0001C66F000EC76F1D
:101DE800020EC86F3F0E4FEC0FF03A0E4FEC11F099
:101DF80012003A0E4FEC11F012003A04D8A4120067
:101E0800010E0001936F375007E10A0E365CD8B017
:101E180003D0364A372A06D0000E376E000E366ECB
:101E2800010E926F355007E1640E345CD8B003D0D0
:101E3800344A352A06D0000E356E000E346E010E77
:101E4800916F000E3A6E12000001CC6F18D0CAC014
:101E5800C7F0CBC0C8F0020E66EC0EF01200CAC084
:101E6800C7F0CBC0C8F0000E66EC0EF01200CAC076
:101E7800C7F0CBC0C8F0010E66EC0EF012000001EE
:101E8800CC51010AD8B4E3D7030AD8B4E8D7010A79
:101E9800D8A41200ECD70001C96F0001C951C009CC
:101EA800CA6F899484B0FED70001CA5140EC10F083
:101EB800000E0001CB6F0DD0CB51010DF350C6259C
:101EC800D96EF450C721DA6ED3EC0FF0DF6E000143
:101ED800CB2BC851CB5DD8A0EFD789841200000165
:101EE800C86F0001C8514009C96F899484B0FED7F2
:101EF8000001C95140EC10F0000E0001CA6F0DD06E
:101F0800CA51010DF350C525D96EF450C621DA6EB9
:101F1800DF5040EC10F00001CA2BC751CA5DD8A0B1
:101F2800EFD7898412000001C36F4C50D8B4FDD795
:101F3800A3B803D0C3C0A9FF12D0A3983F50010D86
:101F4800400EF324D96E010EF420DA6EC3C0DFFF11
:101F58003F2A3F0E3F6402D0000E3F6E4C06A38816
:101F680012000001C66F8FEC11F00001C65169EC38
:101F780011F00001C45169EC11F087EC11F0000177
:101F8800C651010969EC11F09BEC10F00001C56F16
:101F980076EC11F08BEC11F00001C5511200000E27
:101FA8000001C56F000EC46F000EC56F070EC56532
:101FB80001D00FD084A003D0C36BC32B02D0000183
:101FC800C36BC451C425C311C46F8D828D92C52BB8
:101FD800EDD7C45112000BD0C4C0F6FFC5C0F7FF3F
:101FE8000800F55097EC0FF00001C44BC52BC4C096
:101FF800F6FFC5C0F7FF0800F5500009D8A4ECD7D4
:102008000001C605D8A4120062EC11F01200000EFF
:102018000001C36F3B50D8B4FDD73C50010D000EF2
:10202800F324D96E010EF420DA6EDF500001C36F7D
:102038003C2A3F0E3C6402D0000E3C6EA39A3B063D
:10204800A38AC3511200000E396E000E386E000EBE
:10205800376E000E366E000E356E000E346E10ECC4
:1020680011F0CCEC09F093EC11F09EEC0DF083EC40
:1020780011F07FEC11F012000001C36F000E000197
:10208800C46F000EC46F0BD0C3AF02D08D8401D0D3
:102098008D94C351C325C36F8D828D92C42B070EB7
:1020A800C465F2D78D941200400E4C6012D03E5099
:1020B800010D400EF324D96E010EF420DA6EDF50C4
:1020C800A96E3E2A3F0E3E6402D0000E3E6E4C2A98
:1020D8001200A3981200050E0E01DA6F130EF66FA8
:1020E800A89CA88AA898A8849C8E9C9C9C887C867E
:1020F800100EAB6EA49AA38AA498A388A58AA58873
:1021080012009CA202D09C989C883D50010D000EA4
:10211800F324D96E010EF420DA6EAACFDFFF3D2A30
:102128003F0E3D6402D0000E3D6E3B2A1200000EA9
:10213800436E05D0432A0A0E4318D8B402D073B4AC
:10214800F9D70A0E4318D8A402D0FF0E12007186E0
:1021580037EC11F0755012000001C66F8FEC11F0CA
:102168000001C65169EC11F00001C45169EC11F08D
:102178000001C55169EC11F076EC11F08BEC11F00F
:1021880012000001C66F0001C651C009C86F8994CA
:1021980084B0FED70001C85140EC10F0D3EC0FF02A
:1021A8000001C76F8984C75112000001C66F000182
:1021B800C6518009C76F899484B0FED70001C75102
:1021C80040EC10F0D3EC0FF00001C86F8984C851BF
:1021D80012000001C351C503F3CFC7F0F4CFC8F014
:1021E800C351C603F350C827C451C503F350C827C9
:1021F800C7C0C3F0C8C0C4F012000001C66F8994FC
:1022080084B0FED70001C65140EC10F00001C55162
:1022180040EC10F089841200000E3F6E000E3E6EF6
:10222800400E4C6E000E3D6E000E3C6E000E3B6E76
:102238001200B10ED76EE00ED66ED59CD59AD59801
:10224800D586D58EF294F28AF18412003B50D8B428
:1022580012000BEC10F00001C46FC451310AD8B45D
:102268001200030A1200000E436E05D0432A0A0E1C
:102278004318D8B402D09EA6F9D79E961200728A47
:102288007286729472927290000E716E739E739C35
:10229800090E746E12000001C56F899484B0FED7D0
:1022A8000001C55140EC10F08984120030313233FE
:1022B8003435363738394142434445460A0E97EC9F
:1022C8000FF00D0E97EC0FF012000001C36FC3C0A2
:1022D80075FF37EC11F0120080A202D0010E120037
:1022E800000E1200718A718837EC11F012006060DC
:1022F800606060606060340E4FEC11F01200360EC2
:102308004FEC11F01200718237EC11F01200718459
:1023180037EC11F01200718037EC11F01200000E4A
:042328003A6E1200F7
:10FE5E0000436F6E74726F6C426F782056312E3085
:10FE6E0020706F776572656420757020696E205200
:10FE7E0058206D6F64652100202057616974696E8A
:10FE8E0067204D49534F20746F20676F204C4F579A
:10FE9E002E2E2E00202049737375696E67205245F1
:10FEAE0053455420636F6D6D616E642E2E2E005778
:10FEBE00726974696E6720726567697374657273AF
:10FECE002E2E2E00526573657474696E672043433F
:10FEDE00313130312E2E2E0057726974696E6720C3
:10FEEE005041205461626C652E2E2E0050726F634D
:10FEFE00657373696E6720646174612E2E2E0052D5
:10FF0E006563656976696E6720646174612E2E2E55
:10FF1E000054584649464F5F554E444552464C4F45
:10FF2E00570052584649464F5F4F564552464C4F22
:10FF3E005700526164696F2073746174653A2000D2
:10FF4E00545852585F5357495443480052585458C6
:10FF5E005F53574954434800636F6D706C65746509
:10FF6E002E005245474F4E5F4D430056434F4F4E66
:10FF7E005F4D4300535441525443414C00202044A2
:10FF8E006F6E652E0046535F4C4F434B0049464102
:10FF9E0044434F4E004257424F4F53540052585F06
:10FFAE00454E440054585F454E4400454E4443412F
:10FFBE004C004D414E43414C00465354584F4E0059
:10FFCE0052585F525354005245474F4E0056434FBE
:10FFDE004F4E00534C4545500049444C4500584F38
:0AFFEE004646005258005458000027
:08FFF800ACF302FF61F801F017
:00000001FF
